
 Start         Length     Name                   Class
 0001:00401000 0000F130H .text                   CODE
 0002:00411000 000002FCH .itext                  ICODE
 0003:00412000 00000594H .data                   DATA
 0004:00413000 00000058H .bss                    BSS
 0005:00000000 00000000H .tls                    TLS


Detailed map of segments

 0001:00000000 00000216 C=CODE     S=.text    G=(none)   M=System   ACBP=A9
 0001:00000218 00000006 C=CODE     S=.text    G=(none)   M=CheckLst ACBP=A9
 0001:00000220 00000056 C=CODE     S=.text    G=(none)   M=Grids    ACBP=A9
 0001:00000278 0000004E C=CODE     S=.text    G=(none)   M=Mask     ACBP=A9
 0001:000002C8 00000016 C=CODE     S=.text    G=(none)   M=VAUtils  ACBP=A9
 0001:000002E0 000000DC C=CODE     S=.text    G=(none)   M=Windows  ACBP=A9
 0001:000003BC 0000010E C=CODE     S=.text    G=(none)   M=SysUtils ACBP=A9
 0001:000004CC 00000006 C=CODE     S=.text    G=(none)   M=VarUtils ACBP=A9
 0001:000004D4 00000006 C=CODE     S=.text    G=(none)   M=Variants ACBP=A9
 0001:000004DC 00000006 C=CODE     S=.text    G=(none)   M=TypInfo  ACBP=A9
 0001:000004E4 000000BE C=CODE     S=.text    G=(none)   M=Classes  ACBP=A9
 0001:000005A4 00000006 C=CODE     S=.text    G=(none)   M=IniFiles ACBP=A9
 0001:000005AC 00000006 C=CODE     S=.text    G=(none)   M=Registry ACBP=A9
 0001:000005B4 000000B6 C=CODE     S=.text    G=(none)   M=Graphics ACBP=A9
 0001:0000066C 00000006 C=CODE     S=.text    G=(none)   M=UxTheme  ACBP=A9
 0001:00000674 00000006 C=CODE     S=.text    G=(none)   M=MultiMon ACBP=A9
 0001:0000067C 00000006 C=CODE     S=.text    G=(none)   M=DwmApi   ACBP=A9
 0001:00000684 00000006 C=CODE     S=.text    G=(none)   M=HelpIntfs ACBP=A9
 0001:0000068C 00000006 C=CODE     S=.text    G=(none)   M=Printers ACBP=A9
 0001:00000694 00000006 C=CODE     S=.text    G=(none)   M=GraphUtil ACBP=A9
 0001:0000069C 0000005E C=CODE     S=.text    G=(none)   M=ExtCtrls ACBP=A9
 0001:000006FC 00000006 C=CODE     S=.text    G=(none)   M=Clipbrd  ACBP=A9
 0001:00000704 00000006 C=CODE     S=.text    G=(none)   M=FlatSB   ACBP=A9
 0001:0000070C 00000186 C=CODE     S=.text    G=(none)   M=Forms    ACBP=A9
 0001:00000894 0000001E C=CODE     S=.text    G=(none)   M=Menus    ACBP=A9
 0001:000008B4 000002BE C=CODE     S=.text    G=(none)   M=Controls ACBP=A9
 0001:00000B74 00000006 C=CODE     S=.text    G=(none)   M=Themes   ACBP=A9
 0001:00000B7C 00000006 C=CODE     S=.text    G=(none)   M=ActnList ACBP=A9
 0001:00000B84 000000E6 C=CODE     S=.text    G=(none)   M=StdCtrls ACBP=A9
 0001:00000C6C 00000006 C=CODE     S=.text    G=(none)   M=Dialogs  ACBP=A9
 0001:00000C74 00000036 C=CODE     S=.text    G=(none)   M=Buttons  ACBP=A9
 0001:00000CAC 00000006 C=CODE     S=.text    G=(none)   M=ExtDlgs  ACBP=A9
 0001:00000CB4 00000006 C=CODE     S=.text    G=(none)   M=Mapi     ACBP=A9
 0001:00000CBC 00000006 C=CODE     S=.text    G=(none)   M=ExtActns ACBP=A9
 0001:00000CC4 0000008E C=CODE     S=.text    G=(none)   M=ComCtrls ACBP=A9
 0001:00000D54 00000006 C=CODE     S=.text    G=(none)   M=OleCtrls ACBP=A9
 0001:00000D5C 00000006 C=CODE     S=.text    G=(none)   M=AxCtrls  ACBP=A9
 0001:00000D64 00000006 C=CODE     S=.text    G=(none)   M=ComObj   ACBP=A9
 0001:00000D6C 00000006 C=CODE     S=.text    G=(none)   M=OleServer ACBP=A9
 0001:00000D74 00000016 C=CODE     S=.text    G=(none)   M=WinSock  ACBP=A9
 0001:00000D8C 000001C3 C=CODE     S=.text    G=(none)   M=SysInit  ACBP=A9
 0001:00000F50 00000056 C=CODE     S=.text    G=(none)   M=Calendar ACBP=A9
 0001:00000FA8 000003EA C=CODE     S=.text    G=(none)   M=ORDtTmCal ACBP=A9
 0001:00001394 0000006E C=CODE     S=.text    G=(none)   M=ORCtrls  ACBP=A9
 0001:00001404 00000226 C=CODE     S=.text    G=(none)   M=OR2006Compatibility ACBP=A9
 0001:0000162C 0000000E C=CODE     S=.text    G=(none)   M=Rpcconf1 ACBP=A9
 0001:0000163C 00000006 C=CODE     S=.text    G=(none)   M=MFunStr  ACBP=A9
 0001:00001644 00000006 C=CODE     S=.text    G=(none)   M=RpcNet   ACBP=A9
 0001:0000164C 00000046 C=CODE     S=.text    G=(none)   M=Trpcb    ACBP=A9
 0001:00001694 00000006 C=CODE     S=.text    G=(none)   M=Hash     ACBP=A9
 0001:0000169C 00000006 C=CODE     S=.text    G=(none)   M=CCOWRPCBroker ACBP=A9
 0001:000016A4 00000006 C=CODE     S=.text    G=(none)   M=SelDiv   ACBP=A9
 0001:000016AC 00000006 C=CODE     S=.text    G=(none)   M=XWBRich20 ACBP=A9
 0001:000016B4 00000006 C=CODE     S=.text    G=(none)   M=Sgnoncnf ACBP=A9
 0001:000016BC 0000001E C=CODE     S=.text    G=(none)   M=TeEngine ACBP=A9
 0001:000016DC 00000006 C=CODE     S=.text    G=(none)   M=TeCanvas ACBP=A9
 0001:000016E4 00000006 C=CODE     S=.text    G=(none)   M=TeeConst ACBP=A9
 0001:000016EC 00000006 C=CODE     S=.text    G=(none)   M=TeeHtml  ACBP=A9
 0001:000016F4 00000006 C=CODE     S=.text    G=(none)   M=TeeProcs ACBP=A9
 0001:000016FC 00000006 C=CODE     S=.text    G=(none)   M=Chart    ACBP=A9
 0001:00001704 00006780 C=CODE     S=.text    G=(none)   M=ORFn     ACBP=A9
 0001:00007E84 0000147D C=CODE     S=.text    G=(none)   M=ORNet    ACBP=A9
 0001:00009304 00004E42 C=CODE     S=.text    G=(none)   M=ORDtTm   ACBP=A9
 0001:0000E148 00000C1E C=CODE     S=.text    G=(none)   M=ORDtTmRng ACBP=A9
 0001:0000ED68 000003C7 C=CODE     S=.text    G=(none)   M=.ORDateLib2006 ACBP=A9
 0002:00000000 00000006 C=ICODE    S=.itext   G=(none)   M=System   ACBP=A9
 0002:00000008 00000006 C=ICODE    S=.itext   G=(none)   M=CheckLst ACBP=A9
 0002:00000010 00000006 C=ICODE    S=.itext   G=(none)   M=VAUtils  ACBP=A9
 0002:00000018 00000011 C=ICODE    S=.itext   G=(none)   M=Windows  ACBP=A9
 0002:0000002C 00000006 C=ICODE    S=.itext   G=(none)   M=SysUtils ACBP=A9
 0002:00000034 00000006 C=ICODE    S=.itext   G=(none)   M=VarUtils ACBP=A9
 0002:0000003C 00000006 C=ICODE    S=.itext   G=(none)   M=Variants ACBP=A9
 0002:00000044 00000006 C=ICODE    S=.itext   G=(none)   M=TypInfo  ACBP=A9
 0002:0000004C 00000006 C=ICODE    S=.itext   G=(none)   M=Classes  ACBP=A9
 0002:00000054 00000006 C=ICODE    S=.itext   G=(none)   M=IniFiles ACBP=A9
 0002:0000005C 00000006 C=ICODE    S=.itext   G=(none)   M=Registry ACBP=A9
 0002:00000064 00000006 C=ICODE    S=.itext   G=(none)   M=Graphics ACBP=A9
 0002:0000006C 00000006 C=ICODE    S=.itext   G=(none)   M=UxTheme  ACBP=A9
 0002:00000074 00000006 C=ICODE    S=.itext   G=(none)   M=MultiMon ACBP=A9
 0002:0000007C 00000006 C=ICODE    S=.itext   G=(none)   M=DwmApi   ACBP=A9
 0002:00000084 00000006 C=ICODE    S=.itext   G=(none)   M=HelpIntfs ACBP=A9
 0002:0000008C 00000006 C=ICODE    S=.itext   G=(none)   M=Printers ACBP=A9
 0002:00000094 00000006 C=ICODE    S=.itext   G=(none)   M=GraphUtil ACBP=A9
 0002:0000009C 00000006 C=ICODE    S=.itext   G=(none)   M=ExtCtrls ACBP=A9
 0002:000000A4 00000006 C=ICODE    S=.itext   G=(none)   M=Clipbrd  ACBP=A9
 0002:000000AC 00000006 C=ICODE    S=.itext   G=(none)   M=FlatSB   ACBP=A9
 0002:000000B4 00000006 C=ICODE    S=.itext   G=(none)   M=Forms    ACBP=A9
 0002:000000BC 00000006 C=ICODE    S=.itext   G=(none)   M=Menus    ACBP=A9
 0002:000000C4 00000006 C=ICODE    S=.itext   G=(none)   M=Controls ACBP=A9
 0002:000000CC 00000006 C=ICODE    S=.itext   G=(none)   M=Themes   ACBP=A9
 0002:000000D4 00000006 C=ICODE    S=.itext   G=(none)   M=ActnList ACBP=A9
 0002:000000DC 00000006 C=ICODE    S=.itext   G=(none)   M=Dialogs  ACBP=A9
 0002:000000E4 00000006 C=ICODE    S=.itext   G=(none)   M=Buttons  ACBP=A9
 0002:000000EC 00000006 C=ICODE    S=.itext   G=(none)   M=ExtDlgs  ACBP=A9
 0002:000000F4 00000006 C=ICODE    S=.itext   G=(none)   M=Mapi     ACBP=A9
 0002:000000FC 00000006 C=ICODE    S=.itext   G=(none)   M=ExtActns ACBP=A9
 0002:00000104 00000006 C=ICODE    S=.itext   G=(none)   M=ComCtrls ACBP=A9
 0002:0000010C 00000006 C=ICODE    S=.itext   G=(none)   M=OleCtrls ACBP=A9
 0002:00000114 00000006 C=ICODE    S=.itext   G=(none)   M=AxCtrls  ACBP=A9
 0002:0000011C 00000006 C=ICODE    S=.itext   G=(none)   M=ComObj   ACBP=A9
 0002:00000124 00000006 C=ICODE    S=.itext   G=(none)   M=OleServer ACBP=A9
 0002:0000012C 00000008 C=ICODE    S=.itext   G=(none)   M=ORDtTmCal ACBP=A9
 0002:00000134 00000006 C=ICODE    S=.itext   G=(none)   M=ORCtrls  ACBP=A9
 0002:0000013C 00000008 C=ICODE    S=.itext   G=(none)   M=OR2006Compatibility ACBP=A9
 0002:00000144 00000006 C=ICODE    S=.itext   G=(none)   M=Rpcconf1 ACBP=A9
 0002:0000014C 00000006 C=ICODE    S=.itext   G=(none)   M=MFunStr  ACBP=A9
 0002:00000154 00000006 C=ICODE    S=.itext   G=(none)   M=RpcNet   ACBP=A9
 0002:0000015C 00000006 C=ICODE    S=.itext   G=(none)   M=Trpcb    ACBP=A9
 0002:00000164 00000006 C=ICODE    S=.itext   G=(none)   M=Hash     ACBP=A9
 0002:0000016C 00000006 C=ICODE    S=.itext   G=(none)   M=CCOWRPCBroker ACBP=A9
 0002:00000174 00000006 C=ICODE    S=.itext   G=(none)   M=SelDiv   ACBP=A9
 0002:0000017C 00000006 C=ICODE    S=.itext   G=(none)   M=XWBRich20 ACBP=A9
 0002:00000184 00000006 C=ICODE    S=.itext   G=(none)   M=Sgnoncnf ACBP=A9
 0002:0000018C 00000006 C=ICODE    S=.itext   G=(none)   M=TeEngine ACBP=A9
 0002:00000194 00000006 C=ICODE    S=.itext   G=(none)   M=TeCanvas ACBP=A9
 0002:0000019C 00000006 C=ICODE    S=.itext   G=(none)   M=TeeConst ACBP=A9
 0002:000001A4 00000006 C=ICODE    S=.itext   G=(none)   M=TeeHtml  ACBP=A9
 0002:000001AC 00000006 C=ICODE    S=.itext   G=(none)   M=TeeProcs ACBP=A9
 0002:000001B4 00000006 C=ICODE    S=.itext   G=(none)   M=Chart    ACBP=A9
 0002:000001BC 00000090 C=ICODE    S=.itext   G=(none)   M=ORFn     ACBP=A9
 0002:0000024C 00000084 C=ICODE    S=.itext   G=(none)   M=ORNet    ACBP=A9
 0002:000002D0 0000001C C=ICODE    S=.itext   G=(none)   M=ORDtTm   ACBP=A9
 0002:000002EC 00000008 C=ICODE    S=.itext   G=(none)   M=ORDtTmRng ACBP=A9
 0002:000002F4 00000005 C=ICODE    S=.itext   G=(none)   M=.ORDateLib2006 ACBP=A9
 0003:00000000 0000002C C=DATA     S=.data    G=DGROUP   M=SysInit  ACBP=A9
 0003:0000002C 00000510 C=DATA     S=.data    G=DGROUP   M=ORFn     ACBP=A9
 0003:0000053C 0000000E C=DATA     S=.data    G=DGROUP   M=ORNet    ACBP=A9
 0003:0000054C 00000030 C=DATA     S=.data    G=DGROUP   M=ORDtTm   ACBP=A9
 0004:00000000 00000008 C=BSS      S=.bss     G=DGROUP   M=Windows  ACBP=A9
 0004:00000008 0000000C C=BSS      S=.bss     G=DGROUP   M=SysInit  ACBP=A9
 0004:00000014 00000004 C=BSS      S=.bss     G=DGROUP   M=ORDtTmCal ACBP=A9
 0004:00000018 00000008 C=BSS      S=.bss     G=DGROUP   M=OR2006Compatibility ACBP=A9
 0004:00000020 00000010 C=BSS      S=.bss     G=DGROUP   M=ORFn     ACBP=A9
 0004:00000030 00000015 C=BSS      S=.bss     G=DGROUP   M=ORNet    ACBP=A9
 0004:00000048 0000000C C=BSS      S=.bss     G=DGROUP   M=ORDtTm   ACBP=A9
 0004:00000054 00000004 C=BSS      S=.bss     G=DGROUP   M=ORDtTmRng ACBP=A9


  Address             Publics by Name

 0002:000002F4       .ORDateLib2006..ORDateLib2006
 0001:0000F110       .ORDateLib2006.@GetPackageInfoTable
 0001:0000F118       .ORDateLib2006.@PackageLoad
 0001:0000F124       .ORDateLib2006.@PackageUnload
 0004:0000001C       OR2006Compatibility..2
 0001:00001404       OR2006Compatibility..Tfrm2006Compatibility
 0001:000015FC       OR2006Compatibility.Finalization
 0004:00000018       OR2006Compatibility.frm2006Compatibility
 0002:0000013C       OR2006Compatibility.OR2006Compatibility
 0001:000015A8       OR2006Compatibility.Tfrm2006Compatibility.CreateNew
 0004:00000048       ORDtTm..01
 0001:00009BF8       ORDtTm..TORDateBox
 0001:00009844       ORDtTm..TORDateButton
 0001:0000A2F0       ORDtTm..TORDateCombo
 0001:000099AC       ORDtTm..TORDateEdit
 0001:0000970C       ORDtTm..TORDateTimeDlg
 0001:00009E50       ORDtTm..TORDayCombo
 0001:00009304       ORDtTm..TORfrmDtTm
 0001:00009FA4       ORDtTm..TORMonthCombo
 0001:0000A100       ORDtTm..TORYearEdit
 0001:0000A690       ORDtTm.ActiveBroker
 0003:0000054C       ORDtTm.DaysInMonth
 0001:0000C33C       ORDtTm.DaysPerMonth
 0001:0000E118       ORDtTm.Finalization
 0001:0000C2F0       ORDtTm.IsLeapYear
 0001:0000AA14       ORDtTm.LoadEllipsis
 0002:000002D0       ORDtTm.ORDtTm
 0001:0000E09C       ORDtTm.Register
 0001:0000A890       ORDtTm.RelativeDateTime
 0001:0000A6BC       ORDtTm.ServerFMNow
 0001:0000A760       ORDtTm.ServerNow
 0001:0000A7E8       ORDtTm.ServerParseFMDate
 0001:0000A798       ORDtTm.ServerToday
 0001:0000B8D8       ORDtTm.TORDateBox.ButtonClick
 0001:0000BA70       ORDtTm.TORDateBox.Change
 0001:0000B62C       ORDtTm.TORDateBox.Create
 0001:0000C29C       ORDtTm.TORDateBox.GetCaption
 0001:0000C2C0       ORDtTm.TORDateBox.GetDynamicProperty
 0001:0000BAD4       ORDtTm.TORDateBox.GetFMDateTime
 0001:0000BB68       ORDtTm.TORDateBox.GetRelativeTime
 0001:0000C0F8       ORDtTm.TORDateBox.IsValid
 0001:0000BA8C       ORDtTm.TORDateBox.KeyDown
 0001:0000C180       ORDtTm.TORDateBox.SetBlackColorMode
 0001:0000C1C8       ORDtTm.TORDateBox.SetCaption
 0001:0000BC8C       ORDtTm.TORDateBox.SetDateOnly
 0001:0000BDF4       ORDtTm.TORDateBox.SetEditRect
 0001:0000C270       ORDtTm.TORDateBox.SetEnabled
 0001:0000BD3C       ORDtTm.TORDateBox.SetFMDateTime
 0001:0000BD68       ORDtTm.TORDateBox.SetRequireTime
 0001:0000B7EC       ORDtTm.TORDateBox.SetTemplateField
 0001:0000B8BC       ORDtTm.TORDateBox.SupportsDynamicProperty
 0001:0000BE6C       ORDtTm.TORDateBox.UpdateText
 0001:0000BF84       ORDtTm.TORDateBox.Validate
 0001:0000B74C       ORDtTm.TORDateBox.WMSize
 0001:0000D740       ORDtTm.TORDateCombo.BtnClicked
 0001:0000D604       ORDtTm.TORDateCombo.CheckDays
 0001:0000DEB8       ORDtTm.TORDateCombo.CMFontChanged
 0001:0000C3E0       ORDtTm.TORDateCombo.Create
 0001:0000DD24       ORDtTm.TORDateCombo.DateText
 0001:0000D410       ORDtTm.TORDateCombo.DayChanged
 0001:0000C48C       ORDtTm.TORDateCombo.Destroy
 0001:0000DE70       ORDtTm.TORDateCombo.DoChange
 0001:0000DB98       ORDtTm.TORDateCombo.GetFMDate
 0001:0000C508       ORDtTm.TORDateCombo.GetYearSize
 0001:0000C54C       ORDtTm.TORDateCombo.InitDays
 0001:0000C708       ORDtTm.TORDateCombo.InitMonths
 0001:0000D6E8       ORDtTm.TORDateCombo.Loaded
 0001:0000D460       ORDtTm.TORDateCombo.MonthChanged
 0001:0000D714       ORDtTm.TORDateCombo.Paint
 0001:0000C870       ORDtTm.TORDateCombo.Rebuild
 0001:0000DE9C       ORDtTm.TORDateCombo.Resized
 0001:0000CFA4       ORDtTm.TORDateCombo.SetBlackColorMode
 0001:0000CFF8       ORDtTm.TORDateCombo.SetDay
 0001:0000DC18       ORDtTm.TORDateCombo.SetFMDate
 0001:0000D0B4       ORDtTm.TORDateCombo.SetIncludeBtn
 0001:0000D0EC       ORDtTm.TORDateCombo.SetIncludeDay
 0001:0000D148       ORDtTm.TORDateCombo.SetIncludeMonth
 0001:0000D22C       ORDtTm.TORDateCombo.SetLongMonths
 0001:0000D1A4       ORDtTm.TORDateCombo.SetMonth
 0001:0000E0E0       ORDtTm.TORDateCombo.SetTemplateField
 0001:0000D264       ORDtTm.TORDateCombo.SetYear
 0001:0000DEE0       ORDtTm.TORDateCombo.Text
 0001:0000D4B8       ORDtTm.TORDateCombo.YearChanged
 0001:0000DAA8       ORDtTm.TORDateCombo.YearKeyPress
 0001:0000D8FC       ORDtTm.TORDateCombo.YearUDChange
 0001:0000B5FC       ORDtTm.TORDateEdit.CreateParams
 0001:0000B1C0       ORDtTm.TORDateTimeDlg.Create
 0001:0000B22C       ORDtTm.TORDateTimeDlg.Execute
 0001:0000B534       ORDtTm.TORDateTimeDlg.GetFMDateTime
 0001:0000B558       ORDtTm.TORDateTimeDlg.SetDateOnly
 0001:0000B59C       ORDtTm.TORDateTimeDlg.SetFMDateTime
 0001:0000B5D0       ORDtTm.TORDateTimeDlg.SetRequireTime
 0001:0000AAFC       ORDtTm.TORfrmDtTm.calSelectChange
 0001:0000B184       ORDtTm.TORfrmDtTm.cmdCancelClick
 0001:0000AF80       ORDtTm.TORfrmDtTm.cmdMidnightClick
 0001:0000AEE0       ORDtTm.TORfrmDtTm.cmdNowClick
 0001:0000AFB4       ORDtTm.TORfrmDtTm.cmdOKClick
 0001:0000AC74       ORDtTm.TORfrmDtTm.cmdTodayClick
 0001:0000AABC       ORDtTm.TORfrmDtTm.FormCreate
 0001:0000AC04       ORDtTm.TORfrmDtTm.imgNextMonthClick
 0001:0000ABBC       ORDtTm.TORfrmDtTm.imgNextMonthMouseDown
 0001:0000AC4C       ORDtTm.TORfrmDtTm.imgNextMonthMouseUp
 0001:0000ABE4       ORDtTm.TORfrmDtTm.imgPrevMonthClick
 0001:0000AB94       ORDtTm.TORfrmDtTm.imgPrevMonthMouseDown
 0001:0000AC24       ORDtTm.TORfrmDtTm.imgPrevMonthMouseUp
 0001:0000B1A4       ORDtTm.TORfrmDtTm.Loaded
 0001:0000AD28       ORDtTm.TORfrmDtTm.lstHourClick
 0001:0000ADDC       ORDtTm.TORfrmDtTm.lstMinuteClick
 0001:0000ACD8       ORDtTm.TORfrmDtTm.txtTimeChange
 0001:0000C398       ORDtTm.TORYearEdit.SetTemplateField
 0004:0000004C       ORDtTm.uServerToday
 0004:00000014       ORDtTmCal..2
 0001:00000FA8       ORDtTmCal..TORCalendar
 0001:00001364       ORDtTmCal.Finalization
 0002:0000012C       ORDtTmCal.ORDtTmCal
 0001:00001334       ORDtTmCal.Register
 0001:00001138       ORDtTmCal.TORCalendar.DrawCell
 0001:000012C0       ORDtTmCal.TORCalendar.KeyDown
 0004:00000054       ORDtTmRng..3
 0001:0000E37C       ORDtTmRng..TORDateRangeDlg
 0001:0000E148       ORDtTmRng..TORfrmDateRange
 0001:0000ED38       ORDtTmRng.Finalization
 0002:000002EC       ORDtTmRng.ORDtTmRng
 0001:0000EC1C       ORDtTmRng.Register
 0001:0000E5F0       ORDtTmRng.TORDateRangeDlg.Create
 0001:0000E6C0       ORDtTmRng.TORDateRangeDlg.Execute
 0001:0000E940       ORDtTmRng.TORDateRangeDlg.SetDateOnly
 0001:0000EA3C       ORDtTmRng.TORDateRangeDlg.SetFMDateStart
 0001:0000EAA0       ORDtTmRng.TORDateRangeDlg.SetFMDateStop
 0001:0000E9D8       ORDtTmRng.TORDateRangeDlg.SetRequireTime
 0001:0000EB04       ORDtTmRng.TORDateRangeDlg.SetTextOfStart
 0001:0000EB24       ORDtTmRng.TORDateRangeDlg.SetTextOfStop
 0001:0000EC10       ORDtTmRng.TORfrmDateRange.cmdCancelClick
 0001:0000EB44       ORDtTmRng.TORfrmDateRange.cmdOKClick
 0001:0000EC4C       ORDtTmRng.TORfrmDateRange.FormCreate
 0001:0000ECFC       ORDtTmRng.TORfrmDateRange.FormDestroy
 0001:0000ED1C       ORDtTmRng.TORfrmDateRange.Loaded
 0004:00000020       ORFn..1
 0001:000017FC       ORFn..EFMDateTimeError
 0001:000044B8       ORFn..QuickAddError
 0001:00003FE0       ORFn..QuickCopyError
 0001:000076E0       ORFn..TIdleCaller
 0001:00006320       ORFn.AdjustForWindowsXPStyleTitleBar
 0004:00000028       ORFn.AlignList
 0004:0000002C       ORFn.AnchorList
 0001:00005CEC       ORFn.AnchorsToStr
 0001:00004F40       ORFn.BaseFont
 0001:00006DD8       ORFn.BlackColorScheme
 0001:00006EB0       ORFn.BlackColorSchemeUpdate
 0003:0000002C       ORFn.BOOLCHAR
 0001:00007A3C       ORFn.CallWhenIdle
 0001:00007AAC       ORFn.CallWhenIdleNotifyWhenDone
 0001:000025C4       ORFn.CharAt
 0001:00006C9C       ORFn.CheckColorScheme
 0001:000038D8       ORFn.ComparePieces
 0001:00007040       ORFn.ComponentUpdateColorsFor508Compliance
 0001:00002608       ORFn.ContainsAlpha
 0001:000026C0       ORFn.ContainsUpCarretChar
 0001:00002668       ORFn.ContainsVisibleChar
 0001:00002718       ORFn.ConvertSpecialStrings
 0001:000074EC       ORFn.CPRSInstances
 0003:0000011C       ORFn.CRC32_TABLE
 0001:0000283C       ORFn.CRCForFile
 0001:000028EC       ORFn.CRCForStrings
 0001:0000185C       ORFn.DateTimeToFMDateTime
 0001:00003F10       ORFn.DelimCount
 0001:00007C80       ORFn.EnterIsPressed
 0001:00002C04       ORFn.ExpandTabsFilter
 0001:00003054       ORFn.ExtractDefault
 0001:00002F4C       ORFn.ExtractFloat
 0001:00002E50       ORFn.ExtractInteger
 0001:000031FC       ORFn.ExtractItems
 0001:00003398       ORFn.ExtractText
 0001:00004A7C       ORFn.FastAddStrings
 0001:00004944       ORFn.FastAssign
 0004:00000024       ORFn.FBaseFont
 0001:000029F0       ORFn.FilteredString
 0001:00007E00       ORFn.Finalization
 0001:00001BC8       ORFn.FMDateTimeOffsetBy
 0001:00001938       ORFn.FMDateTimeToDateTime
 0001:00005018       ORFn.FontWidthPixel
 0001:00004FA0       ORFn.FontWidthSubPixel
 0001:00005BD0       ORFn.ForceInsideWorkArea
 0001:00001C6C       ORFn.FormatFMDateTime
 0001:0000226C       ORFn.FormatFMDateTimeStr
 0001:00006E18       ORFn.Get508CompliantColor
 0001:00004514       ORFn.GetStrings
 0001:0000403C       ORFn.GetStrings
 0001:000024EC       ORFn.HigherOf
 0003:00000538       ORFn.IdleCaller
 0001:00004D84       ORFn.InfoBox
 0001:00003534       ORFn.InvertStringList
 0001:000022B4       ORFn.IsFMDateTime
 0001:000075EC       ORFn.KillObj
 0001:00004DC8       ORFn.LimitEditWidth
 0001:00004BC0       ORFn.LimitStringLength
 0001:00007230       ORFn.ListGridDrawCell
 0001:00007320       ORFn.ListGridDrawLines
 0001:00007468       ORFn.ListGridRowHeight
 0001:00002514       ORFn.LowerOf
 0001:00004F54       ORFn.MainFont
 0001:00005068       ORFn.MainFontHeight
 0001:00004F88       ORFn.MainFontSize
 0001:00005050       ORFn.MainFontWidth
 0001:0000239C       ORFn.MakeFMDateTime
 0001:00007B20       ORFn.menuHideAllBut
 0001:0000359C       ORFn.MixedCase
 0001:000037B8       ORFn.MixedCaseByPiece
 0001:00003720       ORFn.MixedCaseList
 0003:00000064       ORFn.MONTH_NAMES_LONG
 0003:00000034       ORFn.MONTH_NAMES_SHORT
 0001:00006DF8       ORFn.NormalColorScheme
 0001:000068B0       ORFn.NumCharsFitInWidth
 0002:000001BC       ORFn.ORFn
 0001:00003884       ORFn.Piece
 0001:000038AC       ORFn.Pieces
 0001:00003A58       ORFn.PiecesToList
 0001:00006A04       ORFn.PopupComponent
 0003:00000530       ORFn.PURE_BLACK
 0001:00004874       ORFn.QuickAdd
 0001:000043A0       ORFn.QuickCopy
 0001:00002578       ORFn.RectContains
 0001:000050A8       ORFn.RedrawActivate
 0001:0000508C       ORFn.RedrawSuspend
 0001:00006A58       ORFn.ReformatMemoParagraph
 0003:000000FC       ORFn.ReplaceChars
 0001:000050D0       ORFn.ResetSelectedForList
 0001:0000619C       ORFn.ResizeAnchoredFormToFont
 0001:00005844       ORFn.ResizeChartFonts
 0001:000053F4       ORFn.ResizeCheckListBox
 0001:00005388       ORFn.ResizeComboBox
 0001:00005428       ORFn.ResizeDescendants
 0001:00005A40       ORFn.ResizeFontsInDescendants
 0001:00005FFC       ORFn.ResizeFormToFont
 0001:00005270       ORFn.ResizeHeaderControl
 0001:00005170       ORFn.ResizeHeight
 0001:000053C0       ORFn.ResizeListBox
 0001:000052EC       ORFn.ResizeListView
 0001:000051F0       ORFn.ResizeToFont
 0001:0000511C       ORFn.ResizeWidth
 0001:00005F10       ORFn.RestoreAlign
 0001:00003B04       ORFn.ReverseStr
 0001:000070DC       ORFn.ScanAllComponents
 0003:00000030       ORFn.ScrollBarHeight
 0001:00007D40       ORFn.ScrollControl
 0003:000000DC       ORFn.SearchChars
 0001:00007C98       ORFn.SendMoveMessage
 0001:0000642C       ORFn.SetEqualTabStops
 0001:000023DC       ORFn.SetListFMDateTime
 0001:00003B94       ORFn.SetPiece
 0001:00003CD0       ORFn.SetPieces
 0001:00007C30       ORFn.ShiftTabIsPressed
 0001:00006588       ORFn.ShowMsgOn
 0001:00003DA4       ORFn.SortByPiece
 0001:00006538       ORFn.StatusText
 0001:00005D60       ORFn.StrToAnchors
 0001:0000253C       ORFn.StrToFloatDef
 0001:00005E28       ORFn.SuspendAlign
 0001:00007BE0       ORFn.TabIsPressed
 0001:00006668       ORFn.TextHeightByFont
 0001:000065B8       ORFn.TextWidthByFont
 0001:00007900       ORFn.TIdleCaller.Add
 0001:000078A4       ORFn.TIdleCaller.AppIdle
 0001:00007738       ORFn.TIdleCaller.Create
 0001:00007820       ORFn.TIdleCaller.Destroy
 0001:0000796C       ORFn.TIdleCaller.TimerDone
 0001:00001C00       ORFn.TrimFormatCount
 0003:00000520       ORFn.uBlackColorScheme
 0003:00000534       ORFn.uBorderlessWindowColorWhenBlack
 0003:0000052C       ORFn.uCheckColorScheme
 0003:00000528       ORFn.uMaroonColorWhenBlack
 0003:0000051C       ORFn.uNormalColorScheme
 0001:000071A4       ORFn.UpdateColorsFor508Compliance
 0001:000027B4       ORFn.UpdateCrc32
 0001:000071D4       ORFn.UpdateReadOnlyColorScheme
 0003:00000524       ORFn.uWhiteColorScheme
 0001:00004B3C       ORFn.ValidFileName
 0001:00006728       ORFn.WrappedTextHeightByFont
 0004:00000038       ORNet..1
 0003:0000053C       ORNet.AppStartedCursorForm
 0001:00008C14       ORNet.AuthorizedOption
 0003:00000548       ORNet.BoolChar
 0001:00008B98       ORNet.CallBroker
 0001:000085B0       ORNet.CallBrokerInContext
 0001:00009224       ORNet.CallRPCWhenIdle
 0001:00008FB0       ORNet.CallV
 0001:00008C5C       ORNet.ConnectToServer
 0001:0000917C       ORNet.DottedIPStr
 0001:00007E84       ORNet.EnsureBroker
 0001:00009284       ORNet.Finalization
 0001:00008F54       ORNet.GetRPCCursor
 0001:00009144       ORNet.GetRPCMax
 0001:00008588       ORNet.IsBaseContext
 0001:0000914C       ORNet.LoadRPCData
 0001:00008EF8       ORNet.MRef
 0002:0000024C       ORNet.ORNet
 0001:0000912C       ORNet.RetainedRPCCount
 0004:00000030       ORNet.RPCBrokerV
 0001:000091F0       ORNet.RPCIdleCallDone
 0004:00000034       ORNet.RPCLastCall
 0001:00009004       ORNet.sCallV
 0001:00008BAC       ORNet.SetBrokerServer
 0001:00007EF0       ORNet.SetList
 0001:00007FA8       ORNet.SetParams
 0001:00009138       ORNet.SetRetainedRPCMax
 0001:00009274       ORNet.ShowRPCList
 0001:00009090       ORNet.tCallV
 0003:00000540       ORNet.uBaseContext
 0004:0000003C       ORNet.uCallList
 0003:00000544       ORNet.uCurrentContext
 0004:00000040       ORNet.uMaxCalls
 0001:000084D0       ORNet.UpdateContext
 0004:00000044       ORNet.uShowRPCs
 0001:00000ED4       SysInit.@InitPkg
 0001:00000F38       SysInit.@PackageLoad
 0001:00000F44       SysInit.@PackageUnload
 0001:00000DC4       SysInit.AllocTlsBuffer
 0001:00000E80       SysInit.ExitProcessTLS
 0001:00000E48       SysInit.ExitThreadTLS
 0001:00000D8C       SysInit.FreeLibrary
 0001:00000DD0       SysInit.GetTlsSize
 0004:0000000C       SysInit.HInstance
 0001:00000EA4       SysInit.InitializeModule
 0001:00000E1C       SysInit.InitProcessTLS
 0001:00000DD8       SysInit.InitThreadTLS
 0001:00000D94       SysInit.LocalAlloc
 0001:00000D9C       SysInit.LocalFree
 0003:00000004       SysInit.Module
 0004:00000008       SysInit.ModuleIsLib
 0004:00000009       SysInit.ModuleIsPackage
 0001:00000DA4       SysInit.TlsAlloc
 0004:00000010       SysInit.tlsBuffer
 0001:00000DAC       SysInit.TlsFree
 0001:00000DB4       SysInit.TlsGetValue
 0003:00000000       SysInit.TlsIndex
 0005:00000000       SysInit.TlsLast
 0003:0000001C       SysInit.TlsProc
 0001:00000DBC       SysInit.TlsSetValue
 0001:00000EB0       SysInit.UninitializeModule
 0004:00000000       Windows..3
 0001:000002E8       Windows.CreateFont
 0001:000002F0       Windows.DeleteObject
 0001:00000320       Windows.DrawText
 0001:00000378       Windows.Finalization
 0001:00000328       Windows.FindWindow
 0001:000002E0       Windows.FreeLibrary
 0001:00000330       Windows.GetDC
 0001:000002F8       Windows.GetDeviceCaps
 0001:00000338       Windows.GetKeyState
 0001:00000340       Windows.GetSystemMetrics
 0001:00000300       Windows.GetTextExtentPoint32
 0001:00000308       Windows.GetTextFace
 0001:00000310       Windows.GetTextMetrics
 0001:00000348       Windows.GetWindow
 0001:00000350       Windows.GetWindowText
 0004:00000004       Windows.HtmlHelpModule
 0001:00000358       Windows.InvalidateRect
 0001:00000360       Windows.PtInRect
 0001:00000368       Windows.ReleaseDC
 0001:00000318       Windows.SelectObject
 0001:00000370       Windows.SendMessage
 0002:00000018       Windows.Windows
 0001:00000D7C       WinSock.gethostbyname
 0001:00000D84       WinSock.gethostname
 0001:00000D74       WinSock.inet_ntoa


  Address             Publics by Value

 0001:000002E0       Windows.FreeLibrary
 0001:000002E8       Windows.CreateFont
 0001:000002F0       Windows.DeleteObject
 0001:000002F8       Windows.GetDeviceCaps
 0001:00000300       Windows.GetTextExtentPoint32
 0001:00000308       Windows.GetTextFace
 0001:00000310       Windows.GetTextMetrics
 0001:00000318       Windows.SelectObject
 0001:00000320       Windows.DrawText
 0001:00000328       Windows.FindWindow
 0001:00000330       Windows.GetDC
 0001:00000338       Windows.GetKeyState
 0001:00000340       Windows.GetSystemMetrics
 0001:00000348       Windows.GetWindow
 0001:00000350       Windows.GetWindowText
 0001:00000358       Windows.InvalidateRect
 0001:00000360       Windows.PtInRect
 0001:00000368       Windows.ReleaseDC
 0001:00000370       Windows.SendMessage
 0001:00000378       Windows.Finalization
 0001:00000D74       WinSock.inet_ntoa
 0001:00000D7C       WinSock.gethostbyname
 0001:00000D84       WinSock.gethostname
 0001:00000D8C       SysInit.FreeLibrary
 0001:00000D94       SysInit.LocalAlloc
 0001:00000D9C       SysInit.LocalFree
 0001:00000DA4       SysInit.TlsAlloc
 0001:00000DAC       SysInit.TlsFree
 0001:00000DB4       SysInit.TlsGetValue
 0001:00000DBC       SysInit.TlsSetValue
 0001:00000DC4       SysInit.AllocTlsBuffer
 0001:00000DD0       SysInit.GetTlsSize
 0001:00000DD8       SysInit.InitThreadTLS
 0001:00000E1C       SysInit.InitProcessTLS
 0001:00000E48       SysInit.ExitThreadTLS
 0001:00000E80       SysInit.ExitProcessTLS
 0001:00000EA4       SysInit.InitializeModule
 0001:00000EB0       SysInit.UninitializeModule
 0001:00000ED4       SysInit.@InitPkg
 0001:00000F38       SysInit.@PackageLoad
 0001:00000F44       SysInit.@PackageUnload
 0001:00000FA8       ORDtTmCal..TORCalendar
 0001:00001138       ORDtTmCal.TORCalendar.DrawCell
 0001:000012C0       ORDtTmCal.TORCalendar.KeyDown
 0001:00001334       ORDtTmCal.Register
 0001:00001364       ORDtTmCal.Finalization
 0001:00001404       OR2006Compatibility..Tfrm2006Compatibility
 0001:000015A8       OR2006Compatibility.Tfrm2006Compatibility.CreateNew
 0001:000015FC       OR2006Compatibility.Finalization
 0001:000017FC       ORFn..EFMDateTimeError
 0001:0000185C       ORFn.DateTimeToFMDateTime
 0001:00001938       ORFn.FMDateTimeToDateTime
 0001:00001BC8       ORFn.FMDateTimeOffsetBy
 0001:00001C00       ORFn.TrimFormatCount
 0001:00001C6C       ORFn.FormatFMDateTime
 0001:0000226C       ORFn.FormatFMDateTimeStr
 0001:000022B4       ORFn.IsFMDateTime
 0001:0000239C       ORFn.MakeFMDateTime
 0001:000023DC       ORFn.SetListFMDateTime
 0001:000024EC       ORFn.HigherOf
 0001:00002514       ORFn.LowerOf
 0001:0000253C       ORFn.StrToFloatDef
 0001:00002578       ORFn.RectContains
 0001:000025C4       ORFn.CharAt
 0001:00002608       ORFn.ContainsAlpha
 0001:00002668       ORFn.ContainsVisibleChar
 0001:000026C0       ORFn.ContainsUpCarretChar
 0001:00002718       ORFn.ConvertSpecialStrings
 0001:000027B4       ORFn.UpdateCrc32
 0001:0000283C       ORFn.CRCForFile
 0001:000028EC       ORFn.CRCForStrings
 0001:000029F0       ORFn.FilteredString
 0001:00002C04       ORFn.ExpandTabsFilter
 0001:00002E50       ORFn.ExtractInteger
 0001:00002F4C       ORFn.ExtractFloat
 0001:00003054       ORFn.ExtractDefault
 0001:000031FC       ORFn.ExtractItems
 0001:00003398       ORFn.ExtractText
 0001:00003534       ORFn.InvertStringList
 0001:0000359C       ORFn.MixedCase
 0001:00003720       ORFn.MixedCaseList
 0001:000037B8       ORFn.MixedCaseByPiece
 0001:00003884       ORFn.Piece
 0001:000038AC       ORFn.Pieces
 0001:000038D8       ORFn.ComparePieces
 0001:00003A58       ORFn.PiecesToList
 0001:00003B04       ORFn.ReverseStr
 0001:00003B94       ORFn.SetPiece
 0001:00003CD0       ORFn.SetPieces
 0001:00003DA4       ORFn.SortByPiece
 0001:00003F10       ORFn.DelimCount
 0001:00003FE0       ORFn..QuickCopyError
 0001:0000403C       ORFn.GetStrings
 0001:000043A0       ORFn.QuickCopy
 0001:000044B8       ORFn..QuickAddError
 0001:00004514       ORFn.GetStrings
 0001:00004874       ORFn.QuickAdd
 0001:00004944       ORFn.FastAssign
 0001:00004A7C       ORFn.FastAddStrings
 0001:00004B3C       ORFn.ValidFileName
 0001:00004BC0       ORFn.LimitStringLength
 0001:00004D84       ORFn.InfoBox
 0001:00004DC8       ORFn.LimitEditWidth
 0001:00004F40       ORFn.BaseFont
 0001:00004F54       ORFn.MainFont
 0001:00004F88       ORFn.MainFontSize
 0001:00004FA0       ORFn.FontWidthSubPixel
 0001:00005018       ORFn.FontWidthPixel
 0001:00005050       ORFn.MainFontWidth
 0001:00005068       ORFn.MainFontHeight
 0001:0000508C       ORFn.RedrawSuspend
 0001:000050A8       ORFn.RedrawActivate
 0001:000050D0       ORFn.ResetSelectedForList
 0001:0000511C       ORFn.ResizeWidth
 0001:00005170       ORFn.ResizeHeight
 0001:000051F0       ORFn.ResizeToFont
 0001:00005270       ORFn.ResizeHeaderControl
 0001:000052EC       ORFn.ResizeListView
 0001:00005388       ORFn.ResizeComboBox
 0001:000053C0       ORFn.ResizeListBox
 0001:000053F4       ORFn.ResizeCheckListBox
 0001:00005428       ORFn.ResizeDescendants
 0001:00005844       ORFn.ResizeChartFonts
 0001:00005A40       ORFn.ResizeFontsInDescendants
 0001:00005BD0       ORFn.ForceInsideWorkArea
 0001:00005CEC       ORFn.AnchorsToStr
 0001:00005D60       ORFn.StrToAnchors
 0001:00005E28       ORFn.SuspendAlign
 0001:00005F10       ORFn.RestoreAlign
 0001:00005FFC       ORFn.ResizeFormToFont
 0001:0000619C       ORFn.ResizeAnchoredFormToFont
 0001:00006320       ORFn.AdjustForWindowsXPStyleTitleBar
 0001:0000642C       ORFn.SetEqualTabStops
 0001:00006538       ORFn.StatusText
 0001:00006588       ORFn.ShowMsgOn
 0001:000065B8       ORFn.TextWidthByFont
 0001:00006668       ORFn.TextHeightByFont
 0001:00006728       ORFn.WrappedTextHeightByFont
 0001:000068B0       ORFn.NumCharsFitInWidth
 0001:00006A04       ORFn.PopupComponent
 0001:00006A58       ORFn.ReformatMemoParagraph
 0001:00006C9C       ORFn.CheckColorScheme
 0001:00006DD8       ORFn.BlackColorScheme
 0001:00006DF8       ORFn.NormalColorScheme
 0001:00006E18       ORFn.Get508CompliantColor
 0001:00006EB0       ORFn.BlackColorSchemeUpdate
 0001:00007040       ORFn.ComponentUpdateColorsFor508Compliance
 0001:000070DC       ORFn.ScanAllComponents
 0001:000071A4       ORFn.UpdateColorsFor508Compliance
 0001:000071D4       ORFn.UpdateReadOnlyColorScheme
 0001:00007230       ORFn.ListGridDrawCell
 0001:00007320       ORFn.ListGridDrawLines
 0001:00007468       ORFn.ListGridRowHeight
 0001:000074EC       ORFn.CPRSInstances
 0001:000075EC       ORFn.KillObj
 0001:000076E0       ORFn..TIdleCaller
 0001:00007738       ORFn.TIdleCaller.Create
 0001:00007820       ORFn.TIdleCaller.Destroy
 0001:000078A4       ORFn.TIdleCaller.AppIdle
 0001:00007900       ORFn.TIdleCaller.Add
 0001:0000796C       ORFn.TIdleCaller.TimerDone
 0001:00007A3C       ORFn.CallWhenIdle
 0001:00007AAC       ORFn.CallWhenIdleNotifyWhenDone
 0001:00007B20       ORFn.menuHideAllBut
 0001:00007BE0       ORFn.TabIsPressed
 0001:00007C30       ORFn.ShiftTabIsPressed
 0001:00007C80       ORFn.EnterIsPressed
 0001:00007C98       ORFn.SendMoveMessage
 0001:00007D40       ORFn.ScrollControl
 0001:00007E00       ORFn.Finalization
 0001:00007E84       ORNet.EnsureBroker
 0001:00007EF0       ORNet.SetList
 0001:00007FA8       ORNet.SetParams
 0001:000084D0       ORNet.UpdateContext
 0001:00008588       ORNet.IsBaseContext
 0001:000085B0       ORNet.CallBrokerInContext
 0001:00008B98       ORNet.CallBroker
 0001:00008BAC       ORNet.SetBrokerServer
 0001:00008C14       ORNet.AuthorizedOption
 0001:00008C5C       ORNet.ConnectToServer
 0001:00008EF8       ORNet.MRef
 0001:00008F54       ORNet.GetRPCCursor
 0001:00008FB0       ORNet.CallV
 0001:00009004       ORNet.sCallV
 0001:00009090       ORNet.tCallV
 0001:0000912C       ORNet.RetainedRPCCount
 0001:00009138       ORNet.SetRetainedRPCMax
 0001:00009144       ORNet.GetRPCMax
 0001:0000914C       ORNet.LoadRPCData
 0001:0000917C       ORNet.DottedIPStr
 0001:000091F0       ORNet.RPCIdleCallDone
 0001:00009224       ORNet.CallRPCWhenIdle
 0001:00009274       ORNet.ShowRPCList
 0001:00009284       ORNet.Finalization
 0001:00009304       ORDtTm..TORfrmDtTm
 0001:0000970C       ORDtTm..TORDateTimeDlg
 0001:00009844       ORDtTm..TORDateButton
 0001:000099AC       ORDtTm..TORDateEdit
 0001:00009BF8       ORDtTm..TORDateBox
 0001:00009E50       ORDtTm..TORDayCombo
 0001:00009FA4       ORDtTm..TORMonthCombo
 0001:0000A100       ORDtTm..TORYearEdit
 0001:0000A2F0       ORDtTm..TORDateCombo
 0001:0000A690       ORDtTm.ActiveBroker
 0001:0000A6BC       ORDtTm.ServerFMNow
 0001:0000A760       ORDtTm.ServerNow
 0001:0000A798       ORDtTm.ServerToday
 0001:0000A7E8       ORDtTm.ServerParseFMDate
 0001:0000A890       ORDtTm.RelativeDateTime
 0001:0000AA14       ORDtTm.LoadEllipsis
 0001:0000AABC       ORDtTm.TORfrmDtTm.FormCreate
 0001:0000AAFC       ORDtTm.TORfrmDtTm.calSelectChange
 0001:0000AB94       ORDtTm.TORfrmDtTm.imgPrevMonthMouseDown
 0001:0000ABBC       ORDtTm.TORfrmDtTm.imgNextMonthMouseDown
 0001:0000ABE4       ORDtTm.TORfrmDtTm.imgPrevMonthClick
 0001:0000AC04       ORDtTm.TORfrmDtTm.imgNextMonthClick
 0001:0000AC24       ORDtTm.TORfrmDtTm.imgPrevMonthMouseUp
 0001:0000AC4C       ORDtTm.TORfrmDtTm.imgNextMonthMouseUp
 0001:0000AC74       ORDtTm.TORfrmDtTm.cmdTodayClick
 0001:0000ACD8       ORDtTm.TORfrmDtTm.txtTimeChange
 0001:0000AD28       ORDtTm.TORfrmDtTm.lstHourClick
 0001:0000ADDC       ORDtTm.TORfrmDtTm.lstMinuteClick
 0001:0000AEE0       ORDtTm.TORfrmDtTm.cmdNowClick
 0001:0000AF80       ORDtTm.TORfrmDtTm.cmdMidnightClick
 0001:0000AFB4       ORDtTm.TORfrmDtTm.cmdOKClick
 0001:0000B184       ORDtTm.TORfrmDtTm.cmdCancelClick
 0001:0000B1A4       ORDtTm.TORfrmDtTm.Loaded
 0001:0000B1C0       ORDtTm.TORDateTimeDlg.Create
 0001:0000B22C       ORDtTm.TORDateTimeDlg.Execute
 0001:0000B534       ORDtTm.TORDateTimeDlg.GetFMDateTime
 0001:0000B558       ORDtTm.TORDateTimeDlg.SetDateOnly
 0001:0000B59C       ORDtTm.TORDateTimeDlg.SetFMDateTime
 0001:0000B5D0       ORDtTm.TORDateTimeDlg.SetRequireTime
 0001:0000B5FC       ORDtTm.TORDateEdit.CreateParams
 0001:0000B62C       ORDtTm.TORDateBox.Create
 0001:0000B74C       ORDtTm.TORDateBox.WMSize
 0001:0000B7EC       ORDtTm.TORDateBox.SetTemplateField
 0001:0000B8BC       ORDtTm.TORDateBox.SupportsDynamicProperty
 0001:0000B8D8       ORDtTm.TORDateBox.ButtonClick
 0001:0000BA70       ORDtTm.TORDateBox.Change
 0001:0000BA8C       ORDtTm.TORDateBox.KeyDown
 0001:0000BAD4       ORDtTm.TORDateBox.GetFMDateTime
 0001:0000BB68       ORDtTm.TORDateBox.GetRelativeTime
 0001:0000BC8C       ORDtTm.TORDateBox.SetDateOnly
 0001:0000BD3C       ORDtTm.TORDateBox.SetFMDateTime
 0001:0000BD68       ORDtTm.TORDateBox.SetRequireTime
 0001:0000BDF4       ORDtTm.TORDateBox.SetEditRect
 0001:0000BE6C       ORDtTm.TORDateBox.UpdateText
 0001:0000BF84       ORDtTm.TORDateBox.Validate
 0001:0000C0F8       ORDtTm.TORDateBox.IsValid
 0001:0000C180       ORDtTm.TORDateBox.SetBlackColorMode
 0001:0000C1C8       ORDtTm.TORDateBox.SetCaption
 0001:0000C270       ORDtTm.TORDateBox.SetEnabled
 0001:0000C29C       ORDtTm.TORDateBox.GetCaption
 0001:0000C2C0       ORDtTm.TORDateBox.GetDynamicProperty
 0001:0000C2F0       ORDtTm.IsLeapYear
 0001:0000C33C       ORDtTm.DaysPerMonth
 0001:0000C398       ORDtTm.TORYearEdit.SetTemplateField
 0001:0000C3E0       ORDtTm.TORDateCombo.Create
 0001:0000C48C       ORDtTm.TORDateCombo.Destroy
 0001:0000C508       ORDtTm.TORDateCombo.GetYearSize
 0001:0000C54C       ORDtTm.TORDateCombo.InitDays
 0001:0000C708       ORDtTm.TORDateCombo.InitMonths
 0001:0000C870       ORDtTm.TORDateCombo.Rebuild
 0001:0000CFA4       ORDtTm.TORDateCombo.SetBlackColorMode
 0001:0000CFF8       ORDtTm.TORDateCombo.SetDay
 0001:0000D0B4       ORDtTm.TORDateCombo.SetIncludeBtn
 0001:0000D0EC       ORDtTm.TORDateCombo.SetIncludeDay
 0001:0000D148       ORDtTm.TORDateCombo.SetIncludeMonth
 0001:0000D1A4       ORDtTm.TORDateCombo.SetMonth
 0001:0000D22C       ORDtTm.TORDateCombo.SetLongMonths
 0001:0000D264       ORDtTm.TORDateCombo.SetYear
 0001:0000D410       ORDtTm.TORDateCombo.DayChanged
 0001:0000D460       ORDtTm.TORDateCombo.MonthChanged
 0001:0000D4B8       ORDtTm.TORDateCombo.YearChanged
 0001:0000D604       ORDtTm.TORDateCombo.CheckDays
 0001:0000D6E8       ORDtTm.TORDateCombo.Loaded
 0001:0000D714       ORDtTm.TORDateCombo.Paint
 0001:0000D740       ORDtTm.TORDateCombo.BtnClicked
 0001:0000D8FC       ORDtTm.TORDateCombo.YearUDChange
 0001:0000DAA8       ORDtTm.TORDateCombo.YearKeyPress
 0001:0000DB98       ORDtTm.TORDateCombo.GetFMDate
 0001:0000DC18       ORDtTm.TORDateCombo.SetFMDate
 0001:0000DD24       ORDtTm.TORDateCombo.DateText
 0001:0000DE70       ORDtTm.TORDateCombo.DoChange
 0001:0000DE9C       ORDtTm.TORDateCombo.Resized
 0001:0000DEB8       ORDtTm.TORDateCombo.CMFontChanged
 0001:0000DEE0       ORDtTm.TORDateCombo.Text
 0001:0000E09C       ORDtTm.Register
 0001:0000E0E0       ORDtTm.TORDateCombo.SetTemplateField
 0001:0000E118       ORDtTm.Finalization
 0001:0000E148       ORDtTmRng..TORfrmDateRange
 0001:0000E37C       ORDtTmRng..TORDateRangeDlg
 0001:0000E5F0       ORDtTmRng.TORDateRangeDlg.Create
 0001:0000E6C0       ORDtTmRng.TORDateRangeDlg.Execute
 0001:0000E940       ORDtTmRng.TORDateRangeDlg.SetDateOnly
 0001:0000E9D8       ORDtTmRng.TORDateRangeDlg.SetRequireTime
 0001:0000EA3C       ORDtTmRng.TORDateRangeDlg.SetFMDateStart
 0001:0000EAA0       ORDtTmRng.TORDateRangeDlg.SetFMDateStop
 0001:0000EB04       ORDtTmRng.TORDateRangeDlg.SetTextOfStart
 0001:0000EB24       ORDtTmRng.TORDateRangeDlg.SetTextOfStop
 0001:0000EB44       ORDtTmRng.TORfrmDateRange.cmdOKClick
 0001:0000EC10       ORDtTmRng.TORfrmDateRange.cmdCancelClick
 0001:0000EC1C       ORDtTmRng.Register
 0001:0000EC4C       ORDtTmRng.TORfrmDateRange.FormCreate
 0001:0000ECFC       ORDtTmRng.TORfrmDateRange.FormDestroy
 0001:0000ED1C       ORDtTmRng.TORfrmDateRange.Loaded
 0001:0000ED38       ORDtTmRng.Finalization
 0001:0000F110       .ORDateLib2006.@GetPackageInfoTable
 0001:0000F118       .ORDateLib2006.@PackageLoad
 0001:0000F124       .ORDateLib2006.@PackageUnload
 0002:00000018       Windows.Windows
 0002:0000012C       ORDtTmCal.ORDtTmCal
 0002:0000013C       OR2006Compatibility.OR2006Compatibility
 0002:000001BC       ORFn.ORFn
 0002:0000024C       ORNet.ORNet
 0002:000002D0       ORDtTm.ORDtTm
 0002:000002EC       ORDtTmRng.ORDtTmRng
 0002:000002F4       .ORDateLib2006..ORDateLib2006
 0003:00000000       SysInit.TlsIndex
 0003:00000004       SysInit.Module
 0003:0000001C       SysInit.TlsProc
 0003:0000002C       ORFn.BOOLCHAR
 0003:00000030       ORFn.ScrollBarHeight
 0003:00000034       ORFn.MONTH_NAMES_SHORT
 0003:00000064       ORFn.MONTH_NAMES_LONG
 0003:000000DC       ORFn.SearchChars
 0003:000000FC       ORFn.ReplaceChars
 0003:0000011C       ORFn.CRC32_TABLE
 0003:0000051C       ORFn.uNormalColorScheme
 0003:00000520       ORFn.uBlackColorScheme
 0003:00000524       ORFn.uWhiteColorScheme
 0003:00000528       ORFn.uMaroonColorWhenBlack
 0003:0000052C       ORFn.uCheckColorScheme
 0003:00000530       ORFn.PURE_BLACK
 0003:00000534       ORFn.uBorderlessWindowColorWhenBlack
 0003:00000538       ORFn.IdleCaller
 0003:0000053C       ORNet.AppStartedCursorForm
 0003:00000540       ORNet.uBaseContext
 0003:00000544       ORNet.uCurrentContext
 0003:00000548       ORNet.BoolChar
 0003:0000054C       ORDtTm.DaysInMonth
 0004:00000000       Windows..3
 0004:00000004       Windows.HtmlHelpModule
 0004:00000008       SysInit.ModuleIsLib
 0004:00000009       SysInit.ModuleIsPackage
 0004:0000000C       SysInit.HInstance
 0004:00000010       SysInit.tlsBuffer
 0004:00000014       ORDtTmCal..2
 0004:00000018       OR2006Compatibility.frm2006Compatibility
 0004:0000001C       OR2006Compatibility..2
 0004:00000020       ORFn..1
 0004:00000024       ORFn.FBaseFont
 0004:00000028       ORFn.AlignList
 0004:0000002C       ORFn.AnchorList
 0004:00000030       ORNet.RPCBrokerV
 0004:00000034       ORNet.RPCLastCall
 0004:00000038       ORNet..1
 0004:0000003C       ORNet.uCallList
 0004:00000040       ORNet.uMaxCalls
 0004:00000044       ORNet.uShowRPCs
 0004:00000048       ORDtTm..01
 0004:0000004C       ORDtTm.uServerToday
 0004:00000054       ORDtTmRng..3
 0005:00000000       SysInit.TlsLast


Bound resource files

OR2006Compatibility.dfm
ORDtTm.DFM
ORDtTm.RES
ORDtTmRng.DFM
ORDateLib2006.res
ORDtTm.dcr
ORDtTmRng.dcr
ORDateLib2006.drf


Program entry point at 0002:000002F4
